:1000000009298030A100FE30A7200130A7207530DB
:10001000A7003030BE28A101A117AF00AF08031D13
:100020001328030114280130AF020310A20CA20C04
:10003000A20CC0302205403EAF07FE30A7202F089B
:10004000A728A101A117AF00FE30A7202F08A728DD
:10005000A401AA00AB01A01124080319A0150530C2
:10006000A3002730A900103041200330A900E83058
:100070004120A90164304120A9010A3041202A0809
:100080004828A8002B08A7002A08A600D220260886
:10009000A600A3030319A011240803195228230260
:1000A000031859282608031DA011A0195928303E0D
:1000B000A7280800AD0006118611831606118611C7
:1000C0000F30860583122D08A01884283E30A70023
:1000D0008030BE203330AC0098201330A700883029
:1000E000BE2098206430BD2098206430BD2022308E
:1000F000AC009820283083200C30832006308320E9
:10010000A0142D0884282014AC00201C92288611ED
:10011000033C031C972897200530A700DC30BE2045
:10012000031408002014FE3C0319A5288615201C82
:10013000201006150F3086052C08F03986040611AC
:10014000AC0E201898283230BD202D080429A11BA0
:100150005A2883178001840AFF3E031DAA28042918
:10016000A901A800FF30A807031CA907031C042944
:100170000330A700DF30BE20B228A701E83EA6006A
:10018000A709FC30031CC728A6070318C428A60724
:100190000000A70FC4282618CD28A61CD1280000CF
:1001A000D1280800AB01AA011030AC00270DAA0D20
:1001B000AB0D2808AA022908031C290FAB0203185B
:1001C000E8282808AA0729080318290FAB070310F5
:1001D000A60DA70DAC0BD628260804291030B000B8
:1001E000A701A601AD0CAC0C031CFC282808A6072F
:1001F00029080318290FA707A70CA60CAB0CAA0CFB
:10020000B00BF2282A080429831383120313000079
:100210000800A00107309F00E03083168500FF3002
:1002200086008113831285018601203084006030AE
:10023000AA20A03084005030AA2020308400303022
:10024000A920C830B020012077305A205A205A20E7
:100250002E305A2070305A2069305A2063305A208C
:1002600062305A2061305A2073305A2069305A2047
:1002700063305A202E305A206E305A206C305A206B
:100280000B30A900B830B120012044305A2043304F
:100290005A2046305A2032305A2034305A205530B5
:1002A0005A204B305A2041305A2020305A205A20B0
:1002B00056305A202D305A2032305A200730A900AB
:1002C000D030B120012041305A2064305A206A30A9
:1002D0005A2075305A2073305A2074305A202030FA
:1002E0005A204C305A2044305A2052305A20861816
:1002F0007F29851F7D2905147E2905107729012076
:1003000053305A2065305A2061305A2072305A20BA
:1003100063305A2068305A2020305A2073305A20D7
:1003200069305A2067305A206E305A2061305A2086
:100330006C305A2036140512831605128312232AB4
:10034000C3013C03A500C90149082502031CB929C2
:10035000DC21B61CB7294308A6004908A200A60163
:10036000A20A0314A60DA20BB2292608C304C90FC2
:10037000A429B2014308B100B20CB10CB20CB10C0B
:10038000B20CB10CB20CB10C0F30B2053208AD009A
:100390003108AC00A9010A30A800EE20B1002B08FA
:1003A000B200B4014308B3000F30B3050030B40508
:1003B00031083307C3000800BA01B9010618F12952
:1003C0000130B020B90A0319BA0A0B303A02031CF3
:1003D000F029031DEF29B9303902031CF029B12C93
:1003E000DE299B30B0200618B614061CB610361C49
:1003F0000D2AAD014408AC00A9011830A800EE2078
:10040000B1002B08B2003208A7003108A600A901EC
:100410003A30A800D220BD00162A03013619013E49
:10042000B618013A03193611031D3615C40A85148E
:100430000130A900F430B1208510A901F030A800E6
:100440002808B1200800BB01C4013612361AB12AAF
:10045000BA01B901061C3D2AB90A0319BA0A0130CA
:10046000B020AF303A02031C3C2A031D3B2AC9309E
:100470003902031C3C2AB12C2A2ABA01B9010618F8
:100480006F2AB90A0319BA0A0A30B0203618632A4B
:1004900039080B3A3A04031D4E2A622A3908193AE0
:1004A0003A04031D552A8514622A39084B3A3A0446
:1004B000031D5C2A8510622A3908FA3A3A04031DA2
:1004C000622AB12C6E2A11303A02031C6E2A031DD7
:1004D0006D2A95303902031C6E2AB12C3F2A413017
:1004E0003B02031C742AB12CBB0A3A08031D7C2A68
:1004F00065303902031C7D2A3616361CB02AAD0140
:100500003B08AC00A9011830A800EE20B1002B0870
:10051000B2003208A7003108A600A9014130A800A6
:10052000D220BD008030A1008030212046305A20EA
:100530006F305A2075305A206E305A2064305A205D
:1005400020305A2073305A2069305A2067305A20A0
:100550006E305A2061305A206C305A2020305A2098
:10056000262A361CCD2A012049305A206E305A20C6
:1005700069305A2074305A2069305A2061305A202C
:100580006C305A2069305A207A305A2065305A200F
:100590002E305A205A205A20372B1230BD000130FD
:1005A000A2003D080B20A101B61DE52A3B30410207
:1005B0000318DC2AC10AE42AC101173045020318D6
:1005C000E32AC50AE42AC501E92A4208C10046080F
:1005D000C500051BF92A4508031DF12A0C30C70088
:1005E000F82A0D304502031CF82A0C304502C700DA
:1005F000FE2A4508C70020305A205A200A304702F8
:100600000318042B20305A208030A10047082820EE
:100610003A305A200230A40041082920051B202B23
:100620000C3045020318192B61305A206D305A20C6
:100630001D2B70305A206D305A201530BD00222BF2
:100640001730BD00410803190130031D0301B50037
:100650001E30410203190130031D03013504B500AA
:1006600001308618030135040319372B892C361EF7
:10067000872CDC210130C9000F3049020318432BBD
:10068000DC21C90F3C2B3611B611DC21DC21DC2129
:10069000B61C4C2B05144D2B05101230C90014301C
:1006A00049020318562BDC21C90F4F2BDC210730E0
:1006B000BC00A0214308C200DC21361D602BB6150A
:1006C0000630BC00A0214308C600DC21361D692B82
:1006D000B6150630BC00A0214308BE000330BC00A4
:1006E000A0214308C8000530BC00A0214308C00079
:1006F0000830BC00A0214308BF00DC21361D812B3F
:10070000B615361C872BB619862B36100120B61964
:10071000862C8030A100803021203E082820203007
:100720005A2001304002031DA42B4A305A20613068
:100730005A206E305A2075305A2061305A2072305B
:100740005A2079305A20602C02304002031DB92B08
:1007500046305A2065305A2062305A2072305A2072
:1007600075305A2061305A2072305A2079305A2020
:10077000602C03304002031DC82B4D305A206130DD
:100780005A2072305A2063305A2068305A20602C28
:1007900004304002031DD72B41305A2070305A20BC
:1007A00072305A2069305A206C305A20602C053043
:1007B0004002031DE22B4D305A2061305A2079301F
:1007C0005A20602C06304002031DEF2B4A305A207D
:1007D00075305A206E305A2065305A20602C073010
:1007E0004002031DFC2B4A305A2075305A206C30D1
:1007F0005A2079305A20602C08304002031D0D2CFD
:1008000041305A2075305A2067305A2075305A20AE
:1008100073305A2074305A20602C09304002031D76
:10082000242C53305A2065305A2070305A207430AE
:100830005A2065305A206D305A2062305A20653077
:100840005A2072305A20602C0A304002031D372C87
:100850004F305A2063305A2074305A206F305A205B
:1008600062305A2065305A2072305A20602C0B308A
:100870004002031D4C2C4E305A206F305A207630E7
:100880005A2065305A206D305A2062305A20653027
:100890005A2072305A20602C0C304002031D602C0C
:1008A00044305A2065305A2063305A2065305A202F
:1008B0006D305A2062305A2065305A2072305A20EA
:1008C0000130051B0301B500093040020319013056
:1008D000031D0301350503197A2C20305A202730D7
:1008E0005A208030A1000230A4003F082920203087
:1008F0005A20862C20305A2032305A2030305A204C
:100900008030A1000230A4003F082920882CB12C9F
:10091000232A851F902C0512831605128312922C10
:100920008316051683129B30B0204108031901304D
:10093000031D0301B50001308618030135040319B6
:10094000A22C0515851585140130A900F430B120BD
:100950000511851185100130A9004A30B120C40A63
:100960003A2B01204E305A206F305A2020305A2026
:1009700073305A2069305A2067305A206E305A201E
:1009800061305A206C305A20203084006030AA2018
:10099000A03084005030AA20203084003030A920BC
:1009A0000618B616061CB61203010618013EB61A42
:1009B000013C031DE12CB70A0319B80A0130B0202D
:1009C000D42C0301B61A0130013A0319B612031DE3
:1009D000B61603010618013EB61A013C031DF62C9B
:1009E000B70A0319B80A0130B020E92C03303802E5
:0E09F000DE30031937020318C42C3614232AF4
:02400E00503F21
:00000001FF
